:020000040000FA
:100000008601850107301428030EF0008316850150
:100010008312850190018C01A20A8B010130AF008F
:10002000AD00700E830009009F008923A101831693
:10003000B030860085013730810012309B000C14EF
:1000400083123A3084007923800083169B0A83123E
:10005000840A46300402031D23282017E323B32516
:100060000330A400860085158511A625A40B33282E
:1000700002308600CE252830C0250C30C025063041
:10008000C025E0250321E9010F21691F9028462999
:100090000F212115E0255830C525A401201BA40AF5
:1000A000A01CA40A0330201DA4000430201CA407B7
:1000B000240AC325E625A40D24102408211963234E
:1000C000061E2F23861E33230A3024020319E62836
:1000D00006302402031D8528D0010A30510203187E
:1000E000D1010830510206300319D1000730510206
:1000F00009300319D1000330510206300319D10031
:100100000530510202300319D1004E3051235F26D1
:100110009B250F212119C9230130B425A01B4A2892
:10012000E901861F902803210C3063235108F10058
:100130004030C025EB1C6B18C12FE427F127F727AF
:10014000F727C525E927EF27D027D127C525D027B1
:10015000EA27E627E127E6271330C525EC271930E3
:10016000C525E627C5250630C525F427F427F4273D
:10017000F427E927EF27C525E527F127F727F727F4
:10018000F227C5250330C525F627F527F527F527DE
:10019000F527EF27C525E927F027EA27E527E127F7
:1001A0000A306323F5206C304823E025E9018030D4
:1001B000A4000F21201DAD29A01C502C201F4D2C68
:1001C000A41B042CA40AFF30AC25D928BA25F5209D
:1001D0008D238330CE00C226AC265F2652305123B9
:1001E0004E304823E901652289284E305123523090
:1001F000482387269430CE006C30CF002430D000C6
:10020000D10163270800063063235108EB00080082
:100210006230873C203E243EC525B3250800831666
:10022000F73086008312A6252110A1102111E913B1
:10023000060820067739031D21154339031D2114B3
:100240000139031DA1140608A000A01F6917A11BF6
:100250002D29A01E3221201E36218316B0308600A3
:1002600083120800E9183A2969103C29691C3A29C7
:10027000E9143C296914E910E9170800831685146C
:100280009F0083120730A9259F0808000730C0256A
:100290008730C0250A300A21082147300B2125303C
:1002A0000A215730092108215D300921E825B325AD
:1002B00012300A215F3009211D300A2120300A2125
:1002C00025300A2149300B2108212E300A21E8254A
:1002D000B3250630C025482888306B1D383EC02520
:1002E000EA01861502309F0085303E219F1F6A1467
:1002F000AA303E219F1FEA1486303E219F1F6A15B7
:10030000AB303E219F1FEA15AC303E219F1FEA16FD
:10031000AE303E219F1F6A1707309F0083169F1340
:100320008501831220306A1BC52DEA1A86117118C7
:100330009C296A1C2130C52D00306A180130EA184A
:1003400002306A190330EA190430EA1A7A306A185E
:10035000C52DF20AF2182030C52D2113E9106914B9
:10036000F11820186910E025EB1DC229F525EC25B0
:10037000F0257130C525EA25F025EE25F1257930E7
:10038000C525CD29EB18D929E8256B1CC9293B3097
:10039000CC290030C5256A306E23E8255430E52588
:1003A0008F236918E729E325F6253230C525F12585
:1003B000ED29F525D130E9187B30691C3D30C52584
:1003C0002018E825F625E82584306F218F23E825BD
:1003D0003130C525E918E325F1251030E600632307
:1003E0005108E400D0080319F7295003F829023016
:1003F000E5002018002AA01FA117A11F012ABE2274
:100400008514F925BA250D30EB1C033EE800691868
:10041000132A201C0E2A0430D823C2268D238230B2
:10042000CE00FF26AC265F260430A200E91C222A5B
:100430000310DA0CD90CD80CD70CD60CA20B192A45
:10044000DA0C3E2A69183E2A0310D60DD70DD80DB6
:10045000D90DDA0DA20B242AEA1F302A0530D6075F
:10046000201C3E2A5A0EEB183B2AFF3903193E2A5C
:1004700067150F39031DC3255A08C3256522EB18DC
:10048000492A680B442A462AE825412AA11F6C21E3
:100490004D2AA11B4D2A84306F210F212019612A7A
:1004A000E91BB129A11CF9292018A11FAD29A1130D
:1004B0001208D00050116408D1001030A400C923E4
:1004C000AD29A11392019701D528E918792A590E6F
:1004D000EB1C6719702AFF390319792A0F39031D9C
:1004E000C3255908C325EB187A2A2C30C525E714F3
:1004F0007A2A6714580EEB1CE718832AFF39031970
:10050000872A0F39031DC3255808C3256716570EC0
:10051000EB1C671A8E2A0F390319922AC325EB1C8C
:10052000F625932AE7155708C3259E25201C9E25EE
:10053000E91C9E2A2C30C5255A0EC325EB1CA72A80
:100540008530A11B013EC025A11BB92AAF2AE82591
:10055000E719B12A6B306B184F3E6718B02A4D303F
:10056000C5256B18EB19B92AA130C525E530C5257D
:10057000BC2AF4257A30C525E70108008030C02563
:10058000EA01EB1DCD2A4730C525F025EE25F025E3
:10059000EC25F225EB25ED25EC25EB18D42A43308C
:1005A0006B1C2E3E6E23E825061EDA2A861AE92ADF
:1005B000E403DB2AE40A38230430B425061EE40AE7
:1005C000861EE40338238030AC25061EDE2A861EF4
:1005D000DE2A38238F23A01BF22AFF30E518E5001E
:1005E000E50AB3250130E518103065180430B6006F
:1005F0005F268330EB1C0A3EC0252A30C5259D2589
:100600008316120883126406031D0A2B660865060A
:10061000031908006508E6008F236408831692001A
:100620008312B600B60F152BB50A351C1C2B803073
:10063000950097121712292B171297123608B60732
:10064000361817163610B60C361897163610360CA4
:1006500095006508920012150C3097040800D10A25
:100660000319D00A0800D1080319D003D1030800E8
:100670008F236408B600B60F3E2BB50A8030EB1C02
:100680000A3EC0255F265708C3259D2508003E3039
:10069000A6003330A700542B3330A7004E30532B25
:1006A0005F30A7003330A6000430A2002708840082
:1006B0000008A8002608840028088000A60AA70AC7
:1006C000A20B562B080083169B0083128D237923DF
:1006D000D00083169B0A7923D100080083169B0063
:1006E0001B087923FF3903190800C52583169B0AC7
:1006F000702B83161C141A08831208009B001C150B
:1007000055309D00AA309D009C141C119C18862B0E
:100710000800233084004730922B4E30902B33302A
:1007200084000430A2008001840AA20B932B0800ED
:10073000201BA11AD9282117F925292C523048232A
:10074000502352304D23B4233A304D235B278A2463
:100750003E304D23523051235B278230EB1CC93091
:10076000C025A014CD2CD928C2264C23B230B3000A
:100770006630B4006030B500B130B600FF260230FC
:10078000D823C2268D238A30CE007A30CF00FF26B0
:100790000800500883169A008312240883167E23CB
:1007A0009B0A8312510883169A007F238312080044
:1007B0006323DC23872608002F3048234E30512343
:1007C0002F304D2308000830D8238D23B308031998
:1007D000EE2B8730CE004830CF00FF264C23201F61
:1007E000F62B3E30512363274630FA2B46305123F7
:1007F0005B273E304823B5233A304D23FF26423055
:10080000201B4A3048230800E901E025E825EB1DBC
:10081000182C4330C525F2256C30C525EF256230F4
:10082000C525EC25F225EB25EF25ED25EE251E2C23
:100830001E306B1C2F3EEB187B306E23F925A40174
:100840000930B4258923F9250F214230201F4A3071
:1008500048235F3048230514B3256C210930B425A3
:10086000F925523048234C23051050235B274C2395
:1008700052305123FF260301D823C226211B9E2B71
:100880003E30201F463048234C235023B4233A30B7
:100890004823E32396256C21D928E91C6918552D96
:1008A000E901DE25A01B682C123083169B00831201
:1008B0003A308400000883169A007F239B0A831233
:1008C000840A46300402031D5A2C9625DE25B325E2
:1008D0007730A400A118982BF925A018762CA11E1A
:1008E000742C211BE0252113211BA12B211BE025AA
:1008F00021134C234A30A01C42305123FF268D2364
:100900008130CE005B27B41BE915A018AC2C3A301F
:100910004D23C226E825EB1D9C2C4930C525EE252C
:100920006430C525EA25F1259624A92CEB25F2256E
:10093000EE25F125F0250800EB1CA12C4C30E52517
:10094000A92C31306B1C2F3E6E232C306B1C2F3E9C
:100950006E23A11A8F23CB2C46304D23C226E825C7
:100960004330EB1DBC2CC525F2257030C525F22582
:10097000F125EF259624CC2CEB1CC02CE525CC2CA6
:1009800029306B1C2F3E6E23EB18CC2CE825E82574
:10099000E825E825E825E8256C21A5013308803CF9
:1009A0000318DA2C8D238430CE002030CF00FF26B0
:1009B000A50ACE2C8E30CE001C30CF004030D000A7
:1009C000D101C226AC265F262508B3007530AC00E5
:1009D0007030AB003308031DF72CE325F625A42562
:1009E000A4256919F52CA018392D9E253D2DB30B92
:1009F000072D691DFF2C5708D600D701222DA425ED
:100A0000F625A4259E25A018392D9E253D2DB30B36
:100A1000102D6919ED2CA425A425F6259D253D2D25
:100A2000B30B1A2D6919222DA425A4259E25F62580
:100A30009E253D2D6D30AC006E30AB00B30B262DE6
:100A400069190B2DA425F6259C253D2DE430B30B0B
:100A50002C2D6919142D0B2DB30B322D691D142D5E
:100A60009B25392D2030AC007530AB00B30B0B2D1E
:100A7000512DE919F725E91DE825A018462D2C0868
:100A8000C525F425E825211B0800D9282B0869195C
:100A90007530C525EB1C4E2D211BD928F525E825E1
:100AA000D928A425F6259C253D2D8611E911691527
:100AB00088308B0088306B1D383EC025D730E91850
:100AC000D830C5252030E9188830AC000530E91849
:100AD0001930B4258F238B018E018F0186151014D8
:100AE000851E7B2D0C1C702D0C10B40AAC0B702DC8
:100AF000E6251010D92810100E08B6000F08B50012
:100B000087268D238230CE004030CF005B27B3088C
:100B10000319CD2C0E30D823C2268C30CE001C30C9
:100B2000CF004030D000D101FF26CD2CE0254F3042
:100B3000C525F3250800A425A4259E25563084004C
:100B4000800E0008C325080057309F2D0730AC2DBC
:100B50003F30AE000130AD2DAE01AD00AE0BAE2D7D
:100B6000AD0BAE2D00340230AF00FF30AC25AF0B23
:100B7000B52D080088306B19C02DC030EB1C013E2C
:100B8000A9000511C82D0F393038E803A900051553
:100B9000290ED425851585112908D425851585119B
:100BA00008308605A82500340F39E300E3196317E0
:100BB000E3118619E3156308860008000230E12D71
:100BC0000130C025A62D3030C52DC5253D30C52DA1
:100BD0002030C52D013E023E033E013E053E043E4F
:100BE000023E023E163E033E023E183E013E2D3EB0
:100BF000C52D88308B00A2016C3051238D23E91C58
:100C0000062ECF168430CE00C2260C2E69180C2E6C
:100C1000CF168330CE00FF26AC263408A30035085B
:100C2000FF3C8F0036086918172E043C182E053C2F
:100C30008E00B9188E038F23900A8316051683122F
:100C400081010B1D2A2EFF30031134020319B30A50
:100C5000B40A0B112218332E0C1C212E0C10A30BDE
:100C6000212E0B17212E0B1D3C2EFF3003113402B9
:100C70000319B30AB40A0B110108B500B601B60A8C
:100C800083160116432E01128312462E010803110A
:100C9000350203193F2EB609B60A0B113618EA17AA
:100CA000A112F0303605350434040319A116691871
:100CB00008008726201D08004C23C226080020308B
:100CC000AE00D601D701D801D901DA01B60DB50DB4
:100CD000B40DB30DD60DD70DD80DD90DDA0DAE0B61
:100CE000722E08000530A30056308400782E840A46
:100CF0007C26A30B772E662E03300007AD00AD19BE
:100D0000800030300007AD00AD1B80000800983037
:100D1000B300AA01AD013408031D9F2E3508B400AD
:100D20003608B500B601AD153408031D9F2E3508F1
:100D3000B400B501AD112D1634080319C02E2D08CD
:100D4000B3020310B41BA92EB60DB50DB40DB30339
:100D5000A22EAA1FB413003432304823B601B317B1
:100D60008030B202B21F0319C02E3208203CB200FC
:100D70000310B30CB40CB50CB60CB20BB82E003487
:100D80008F2300343308031D4E080319C02E340886
:100D90004F06AA004E08B3078030031CD12EB307BC
:100DA000D22EB307B417CF170310B701B801B9019A
:100DB0001830AD00361CE62E5108B907500803184C
:100DC000500FB8074F0803184F0FB707B70CB80CF0
:100DD000B90CB40CB50CB60C0310AD0BDA2EB71B66
:100DE000F62EB40DB90DB80DB70DB303AA1FB71386
:100DF0003708B4003808B5003908B60000343408A4
:100E00004F06AA00B417CF17AD013408B700350854
:100E1000B8003608B9005108B9025008031C500F39
:100E2000B8024F08031C4F0FB702B701B801B90150
:100E3000031C212F0310B40CB50CB60CB70C0130F9
:100E4000AD004E08B302031C292F80302D07B307D5
:100E50002C2F80302D07B3071830AE00B90DB80D18
:100E6000B70DB60DB50DB40DAD0D5108B602500855
:100E7000031C500FB5024F08031C4F0FB4024F0D57
:100E8000AD042D1C452F3914502F5108B6075008BA
:100E90000318500FB5074F0803184F0AB40739104D
:100EA000AE0B2E2FAA1FB7133708B4003808B500B1
:100EB0003908B60000344E08031D612F4F0803198E
:100EC00000348030CF0634084F06AD0033084E02A0
:100ED000031C6B2FDC233408AA00B417CF174F086C
:100EE000B7005008B8005108B9004E083302CE00D0
:100EF0000319972F08304E02031C8E2FCE00B90D18
:100F00003808B9003708B800B70108304E02031C92
:100F10008E2FCE00B90D3808B900B8014E0803195C
:100F2000972F0310B70CB80CB90CCE0B912FAD1F37
:100F3000A12FB709B809B909B90A0319B80A0319E1
:100F4000B70A3908B60738080318380FB507370845
:100F50000318370FB407AD1BB42F031CA92EB40C14
:100F6000B50CB60CB30AA92E03188A2EB409B5091C
:100F7000B609B60A0319B50A0319B40A8030AA06DD
:100F80008A2ED427D727E127D427D827E027D427AC
:100F9000D927DF27D427EE27DE27F327DC27D02821
:100FA000F027F027F0270800F327EA270800EE27AC
:100FB000EE27EE27EE270800EA27EA27EA27EA27A6
:100FC000EA27EA27C5250800EF27EF27EF27EF27B5
:100FD0000800013E073E023E013E023E013E013E48
:100FE000013E013E023E023E013E043E043E013E01
:0C0FF000C52D2030563032302E30343009
:02400E00013F70
:10420000040039000300E800000040000000000046
:104210000000000080000000000000000000C80056
:104220000100F90086006A008D00A0008A000900E4
:10423000E400F800A3006900660099004B006100EB
:10424000BB00B800B20070006F00B300BA0061009C
:104250000000A200BC00BA006F006300BF00C400F1
:104260000000A500BD00E3007900BA00BF00B8005F
:10427000B300BD000000AB0061006300BF006F0031
:10428000BF0061000000A1006500BD006500700076
:104290006100BF006F00700000004B00410006008D
:1042A0000300070050004F0042004B004100000097
:1042B00045004D004B004F00430054000200000039
:1042C00003004800040005004B00540003004200B6
:1042D000480000004100430054004F0054004100DA
:1042E0000000010045004800450050004100540016
:1042F0004F0050000000570061006900740000008A
:00000001FF
